:020000040000FA
:10000000052800000000000000008501860183161D
:10001000850186018312FF3085008600132085014B
:10002000860113200B2803308E0089308D008C0B45
:1000300017288D0B17288E0B17280800FF3FFF3F4E
:10004000FF3FFF3FFF3FFF3FFF3FFF3FFF3FFF3FC0
:10005000FF3FFF3FFF3FFF3FFF3FFF3FFF3FFF3FB0
:10006000FF3FFF3FFF3FFF3FFF3FFF3FFF3FFF3FA0
:10007000FF3FFF3FFF3FFF3FFF3FFF3FFF3FFF3F90
:02400E00F13F80
:08400000FF3F0F000F000F004D
:00000001FF
